:0600000000308A002D28EB
:10000800F50003088301C5000408C6000A08C700F4
:100018008A017008C8007108C9008B180B1E1828BF
:10002800F32370083F39B0000B188B1D1C280726D6
:080038008B100B10031383125F
:100040004808F0004908F1004608840047088A0083
:1000500045088300F50E750E0900203084004530F8
:100060003520112D04068001840A0406031D322860
:1000700064000034F000F4010310FD307107031C2C
:100080006128F301F0307105031D49280430F300A5
:10009000F10EF2010310F30AF10D031C4B28F10CD1
:1000A000710870020318F000F20DF30B4F28F41FD3
:1000B0005B28F209F20A7208F41F0800F009F00A3E
:1000C0000800F10C03186A28F10C031CF00103105E
:1000D000F00C031C03107008F200F001F00D57281B
:1000E0008301B700723A031DAD28783083169B0058
:1000F0001C141A088312AF00793083169B001C145D
:100100001A088312A3007A3083169B001C141A0865
:100110008312A4007B3083169B001C141A088312E0
:10012000AC007C3083169B001C141A088312A700B5
:100130007D3083169B001C141A088312A5007E30A4
:1001400083169B001C141A088312AA007F308316A2
:100150009B001C141A088312AB003708773A031D62
:100160005A2983169C18B12878309B0083122F08D7
:1001700083169A0003108B1B03148B131C15553028
:100180009D00AA309D009C141C1103188B179C180D
:10019000C72879309B008312230883169A00031026
:1001A0008B1B03148B131C1555309D00AA309D002A
:1001B0009C141C1103188B179C18DC287A309B00A8
:1001C0008312240883169A0003108B1B03148B13CD
:1001D0001C1555309D00AA309D009C141C1103185D
:1001E0008B179C18F1287B309B0083122C088316F8
:1001F0009A0003108B1B03148B131C1555309D00A4
:10020000AA309D009C141C1103188B179C180629FA
:100210007C309B008312270883169A0003108B1BE7
:1002200003148B131C1555309D00AA309D009C149F
:100230001C1103188B179C181B297D309B008312FF
:10024000250883169A0003108B1B03148B131C15AF
:1002500055309D00AA309D009C141C1103188B176B
:100260009C1830297E309B0083122A0883169A003E
:1002700003108B1B03148B131C1555309D00AA30E3
:100280009D009C141C1103188B179C1845297F3066
:100290009B0083122B0883169A0003108B1B0314F8
:1002A0008B131C1555309D00AA309D009C141C1109
:1002B00003188B17831208008B1383120313201B60
:1002C000322A32083104031967292908A8000730A7
:1002D0002802031C6D29A801A80A0130280203186E
:1002E00073290630A800B701B70A28084724280B4D
:1002F0008C292808290603197F292F08AD002D0F06
:100300008229AD0149302D02031C88294830AD00F7
:100310002D0846262D08AF002808023A031DA629FD
:1003200028082906031996292308AD0001302D025B
:1003300003189C29AD01AD0A41302D02031CA229EE
:100340004030AD002D08E7252D08A3002808033A0A
:10035000031DBD29280829060319B0292408AD006A
:100360002D0FB329AD0110302D02031CB9290F3018
:10037000AD002D08A8262D08A4002808043A031D66
:10038000D429280829060319C7292C08AD002D0FE8
:10039000CA29AD0110302D02031CD0290F30AD0049
:1003A0002D08A8262D08AC002808053A031DF829B9
:1003B000320831040319DE292E08AD002808290669
:1003C0000319E4292708AD00AD08031DE92904300D
:1003D000AD0005302D02031CEF29AD01AD0A2D083B
:1003E00070250230B70028082D0747242D08A700E4
:1003F0002808063A031D222A320831040319022A6A
:100400002E08AD00280829060319082A2508AD0082
:10041000AD08031D0D2A0230AD0003302D02031C70
:10042000132AAD01AD0AB701B70A2808043E4724D4
:100430002D0870250230B7002D082807043E4724F8
:100440002D08A500A01A262A7730272A723070209E
:100450002808A9002D08AE00FF30B300B400B10099
:100460000830B20035228B170800C6308301B8006F
:10047000A01E3C2A2030B807201F402A2030B80791
:10048000270B442A0830B8072708023A031D4A2AD6
:100490001830B8072708033A031D502A1030B80750
:1004A0002508023A0319B80A03102F0CB7002130AF
:1004B0002302031C6A2AFB30F000F1012308F0023A
:1004C000031CF1033708F0070318F10A7008B9009C
:1004D0007108732ADB30F000F10137087007B900AA
:1004E00071080318710ABA00203023020318872A02
:1004F0002308F000F1013708F0070318F10ABB30B8
:100500007007BB000030031801307107902ADB3000
:10051000F000F10137087007BB0071080318710A79
:10052000BC0000303A02DB300319390203189B2A61
:10053000DB30B900BA0101303A0200300319390248
:10054000031CA52AFF30B900BA0100303C02DB30A1
:1005500003193B020318AF2ADB30BB00BC0101309A
:100560003C02003003193B02031CB92AFF30BB00D8
:10057000BC01D0268230C5250030C5253908C525E7
:100580003B08C5252408F03EC5252C08F03EC525AE
:10059000D0268230C5250830C5253808C525042F4A
:1005A000830128030319DB2A34083304031DDB2AE3
:1005B000A801A80A5C21B008031908008B132608BB
:1005C0003006031D392B3008203A031DE92AA80AFA
:1005D0005C213008213A031DEF2AA8035C21300872
:1005E000103A0319F72A3008163A031DF92AAD0A02
:1005F0005C213008113A0319012B3008153A031D0C
:10060000032BAD035C213008173A031D0A2BA80108
:10061000A80A5C2130082B3A031D112B0230A800D8
:100620005C2130082C3A031D182B0330A8005C21F4
:1006300030082D3A031D1F2B0430A8005C21300820
:100640002E3A031D262B0530A8005C213008383ACD
:1006500003192E2B3008233A031D312B0630A80036
:100660005C2130080D3A0319792630080C3A031939
:10067000E4263008A600B0018B1708008301BD00F6
:10068000A200220D220D0139F000700C031C4A2B30
:1006900005174B2B0513220EF000F00C700C0139DE
:1006A000F000700C031C562B8517572B8513220E58
:1006B000F000700C0139F000700C031C612B051464
:1006C000622B0510220E0139F000700C031C6A2BFE
:1006D00085146B2B85100F27220CF000F00C700C8A
:1006E0000139F000700C031C772B0517782B0513CC
:1006F000220CF000700C0139F000700C031C822BEE
:100700008517832B8513220C0139F000700C031C14
:100710008B2B05148C2B051022080139F000700C6E
:10072000031C942B8514952B85100F27ED26201B79
:100730009B2B0516080005120800830105117F3068
:100740003E23051500303E2304303E230A303E236D
:1007500011303E2311303E2315303E230A303E2314
:1007600000303E2301303E2303303E231D303E2324
:1007700015303E231D303E2303303E2301303E23FF
:1007800000303E2310303E2318303E2317303E23E6
:1007900015303E2317303E2318303E2310303E23C1
:1007A00000303E23B6011E303E23B60A0830360222
:1007B000031CD32BB6011C303E23B60A0830360288
:1007C000031CDB2BB60118303E23B60A0830360274
:1007D000031CE32BB60110303E23B60A0830360264
:1007E00003180800EB2B8301C101C2010618422C3B
:1007F000C0014208F1004108F0000310F00DF10DB6
:100800000030061801307007C10071080318710A22
:10081000C200A430C300C4010000FF30C307031CA2
:10082000C40344084304031D0C2C00300618013097
:10083000BF003230C300C4010000FF30C307031CF7
:10084000C4033F08F000F1010030061801307006C3
:100850007104003003190130F000F1014308F00584
:100860004408F10571087004031D1C2C440843045E
:10087000031D3D2CF001F1010800C00A0E304002BA
:10088000031CF92B4208F1004108F0000800830125
:10089000B80037089C25BA013A0883169B001C143F
:1008A0001A0883123806031D782CBA0AB9013A08CF
:1008B00083169B001C1483123808F000F1010130EC
:1008C000F0070318F10A83161A08700671048312E0
:1008D0000319712C3A0883169B001C141A083E2336
:1008E000BA0AB90A10303902031C572C8030BA00FA
:1008F000BA0A80303A02031808004C2C4125A1089E
:1009000003190800210B852CE4262108033A03195A
:1009100079262108043A031D8F2CAD035C212108A0
:10092000063A031D952CAD0A5C212108023A031DED
:100930009B2CA80A5C212108053A031DA12CA803C1
:100940005C21A101FF30B5000F30B6000000350872
:100950000319B603B503350A0319360A031908004B
:10096000A62C47303E2399264F303E2399264F3000
:100970003E23992644303E23992620303E234230A0
:100980003E23992659303E23992645303E23992609
:100990002C303E23992620303E2342303E23992698
:1009A00041303E23992642303E23992659303E233A
:1009B000992620303E2321303E23992699269926D8
:1009C000992E07303E23992620303E2324303E23A3
:1009D000992659303E23992650303E23992645309A
:1009E0003E23992652303E23992620303E234E3016
:1009F0003E23992641303E23992624303E239926D2
:100A000054303E23992659303E23992641303E23C7
:100A1000992620303E2307303E2399269926992691
:100A2000992EFF3083120313B300B4000000330883
:100A30000319B403B303330A0319340A031D162D33
:100A4000652627267230702016278B17201B2A2D2B
:100A500005162B2D051283120313320831040319D6
:100A6000352DB1080319B203B10334083304031957
:100A70003D2DB3080319B403B303D022B7267E2457
:100A8000262D8B13831203130510861B492DA101FC
:100A9000A10A061B4D2D0230A100861A512D0330EC
:100AA000A10005148513861B572D0430A100061BD9
:100AB0005B2D0530A100861A5F2D0630A100851739
:100AC0000513861B652D0730A100061B692D083014
:100AD000A100861A6D2D0930A10005178B1708009B
:100AE0008301BC00BA01BB01B90105118E303E2360
:100AF0000515A01E7F2D982DBA0A9C30BC076430C6
:100B00003C02031C872D7C2DBB0AF630BC070A3043
:100B10003C020318842D3C08B900BB080319932D2F
:100B20003B08303E942D20303E233908303E3E2B8A
:100B300078303E2305303E2B8301BB003B0BB02DAC
:100B4000051180303E230515BC0120303E23BC0A30
:100B500010303C02031CA52D051180303E230515E5
:100B60003B08023A031D08000511C0303E2305155D
:100B7000BC0120303E23BC0A10303C02031CB92DBE
:100B80000511C0303E23051508008301BD00083063
:100B9000BE00DE2DBE033D08F0003E08F100F10A64
:100BA000D32D0310F00CF10BD12D7008F000700C58
:100BB000031CDC2D0615DD2D0611FE26BE08031DC7
:100BC000CA2D00008301FE26000083010800830176
:100BD000B70002309C25B801FF303E23B80A103020
:100BE0003802031CEC2D05113708F0000310F00C3F
:100BF0000310700CBF3E3E23051502303702031C64
:100C0000032E05303E2306303E233708702D830126
:100C1000A010061AA014201186192015201D122ECE
:100C20000130132E0030F000A01D182E0130192EB7
:100C30000030F006031D2019232EA018212E2012AB
:100C4000222E20162014A0112019A01508008301BF
:100C5000B501ED26B50A8F303502031C292E05118A
:100C600005138513051485100F27B501ED26B50A68
:100C700027303502031C362E2B303E2313303E2303
:100C80000C303E2304303E239D23892E8301B70080
:100C900002309C25B8014F2EFF303E23B80A0530A4
:100CA000F10037083A203802031C4C2E0530F100C1
:100CB0003808C4263702B800B808031D612E20305A
:100CC000B80038083E233708702D8B0183160313B4
:100CD0008501F9308600073083129F008501860167
:100CE000831681130B168B1001138B150B108312B7
:100CF0000800830132083104031D842EA01A822EBD
:100D0000A016832EA0125C21FF30B1000830B20083
:100D100008008301051101303E23B701ED26B70A13
:100D200013303702031C8E2E051180303E2305152B
:100D300008008301B701B8010000B70A0319B80A17
:100D40004F303802FF3003193702031808009C2E79
:100D50008301B70002309C25B801B12EFF303E233D
:100D6000B80A37083802031CAE2E3708702D8301ED
:100D7000201C08008B13201EBF2EAD0AC02EAD0311
:100D80005C2120108B170800F000003071187007EC
:100D90000310F00D0310F10CF10803190800C62E22
:100DA00083010615861400008301061100008301EB
:100DB000861008008301051107303E231C303E23B6
:100DC0008F303E23051508008301201BEA2E2017D3
:100DD0000A275C29201316275C298301BE01000025
:100DE000BE0A0C303E0203180800EF2E83010511E5
:100DF00013303E2304303E2305150800830186147A
:100E0000000083018610080083018614000083011E
:100E1000061508008926DA26B124F626892E8301D4
:100E20008515851108000000830108008926E12C42
:02400E00503F21
:104200000100A10070006F00BC00BA006F006300E5
:10421000BF00C4000200A0006100BB006100BD003F
:104220006300030054006500BC00B2007000200071
:10423000BD00B800B700BA00B80065000400540023
:104240006500BC00B20070002000B300C300630032
:104250006F00BA00B8006500050050006500B600A8
:10426000B800BC0006006F00B200C300C000BD0073
:10427000C300B9000700700061006300C100B8000E
:1042800070006500BD00BD00C300B9000800BE009D
:1042900063006500B300E3006F006300BF006500CA
:1042A000700065006F000900BC006F00BD006F006A
:1042B0000A00420078006F00E3000B00BB00B8006A
:1042C000BD006500B900BD00C300B9000C00BE0010
:1042D0007000B800B500BC00BD00B800BA000D0009
:1042E0004E006100730074007900610020000E0030
:1042F000210020000800080001000100000000006B
:00000001FF
